ARM Linker, 5.03 [Build 76] [MDK-ARM Lite]

==============================================================================

Section Cross References

    hhd_sys.o(.text) refers to system_hhd32f0xx.o(.text) for SystemInit
    hhd_sys.o(.text) refers to hhd_sys.o(i.__ARM_common_switch8) for __ARM_common_switch8
    hhd_uart.o(.text) refers to aeabi_sdiv.o(.text) for __aeabi_uidivmod
    hhd_uart.o(.text) refers to system_hhd32f0xx.o(.data) for MainClock
    hhd_iic.o(.text) refers to aeabi_sdiv.o(.text) for __aeabi_uidivmod
    hhd_iic.o(.text) refers to system_hhd32f0xx.o(.data) for SystemCoreClock
    hhd_iic.o(.text) refers to hhd_iic.o(.data) for IICMasterState
    system_hhd32f0xx.o(.text) refers to aeabi_sdiv.o(.text) for __aeabi_uidivmod
    system_hhd32f0xx.o(.text) refers to system_hhd32f0xx.o(.data) for MainClock
    startup_hhd32f0xx_s.o(STACK) refers (Special) to heapauxi.o(.text) for __use_two_region_memory
    startup_hhd32f0xx_s.o(HEAP) refers (Special) to heapauxi.o(.text) for __use_two_region_memory
    startup_hhd32f0xx_s.o(RESET) refers (Special) to heapauxi.o(.text) for __use_two_region_memory
    startup_hhd32f0xx_s.o(RESET) refers to startup_hhd32f0xx_s.o(STACK) for __initial_sp
    startup_hhd32f0xx_s.o(RESET) refers to startup_hhd32f0xx_s.o(.text) for Reset_Handler
    startup_hhd32f0xx_s.o(.text) refers (Special) to heapauxi.o(.text) for __use_two_region_memory
    startup_hhd32f0xx_s.o(.text) refers to __main.o(!!!main) for __main
    startup_hhd32f0xx_s.o(.text) refers to startup_hhd32f0xx_s.o(HEAP) for Heap_Mem
    startup_hhd32f0xx_s.o(.text) refers to startup_hhd32f0xx_s.o(STACK) for Stack_Mem
    main.o(.text) refers to hhd_sys.o(.text) for SYS_SystemInitial
    main.o(.text) refers to hhd_iic.o(.text) for IIC_Init
    main.o(.text) refers to hhd_uart.o(.text) for UART_Open
    main.o(.text) refers to at24c02.o(.text) for AT24C02_WriteBYTE
    lm75a.o(.text) refers to hhd_iic.o(.text) for IIC_ReadArray
    sd2405alpi.o(.text) refers to hhd_iic.o(.text) for IIC_ReadByte
    at24c02.o(.text) refers to hhd_iic.o(.text) for IIC_ReadByte
    __main.o(!!!main) refers to rtentry.o(.ARM.Collect$$rtentry$$00000000) for __rt_entry
    rtentry.o(.ARM.Collect$$rtentry$$00000000) refers (Special) to rtentry2.o(.ARM.Collect$$rtentry$$0000000A) for __rt_entry_li
    rtentry.o(.ARM.Collect$$rtentry$$00000000) refers (Special) to rtentry2.o(.ARM.Collect$$rtentry$$0000000D) for __rt_entry_main
    rtentry.o(.ARM.Collect$$rtentry$$00000000) refers (Special) to rtentry2.o(.ARM.Collect$$rtentry$$0000000C) for __rt_entry_postli_1
    rtentry.o(.ARM.Collect$$rtentry$$00000000) refers (Special) to rtentry2.o(.ARM.Collect$$rtentry$$00000009) for __rt_entry_postsh_1
    rtentry.o(.ARM.Collect$$rtentry$$00000000) refers (Special) to rtentry2.o(.ARM.Collect$$rtentry$$00000002) for __rt_entry_presh_1
    rtentry.o(.ARM.Collect$$rtentry$$00000000) refers (Special) to rtentry4.o(.ARM.Collect$$rtentry$$00000004) for __rt_entry_sh
    aeabi_idiv0_sigfpe.o(.text) refers to rt_div0.o(.text) for __rt_div0
    rtentry2.o(.ARM.Collect$$rtentry$$00000008) refers to boardinit2.o(.text) for _platform_post_stackheap_init
    rtentry2.o(.ARM.Collect$$rtentry$$0000000A) refers to libinit.o(.ARM.Collect$$libinit$$00000000) for __rt_lib_init
    rtentry2.o(.ARM.Collect$$rtentry$$0000000B) refers to boardinit3.o(.text) for _platform_post_lib_init
    rtentry2.o(.ARM.Collect$$rtentry$$0000000D) refers to main.o(.text) for main
    rtentry2.o(.ARM.Collect$$rtentry$$0000000D) refers to exit.o(.text) for exit
    rtentry2.o(.ARM.exidx) refers to rtentry2.o(.ARM.Collect$$rtentry$$00000001) for .ARM.Collect$$rtentry$$00000001
    rtentry2.o(.ARM.exidx) refers to rtentry2.o(.ARM.Collect$$rtentry$$00000008) for .ARM.Collect$$rtentry$$00000008
    rtentry2.o(.ARM.exidx) refers to rtentry2.o(.ARM.Collect$$rtentry$$0000000A) for .ARM.Collect$$rtentry$$0000000A
    rtentry2.o(.ARM.exidx) refers to rtentry2.o(.ARM.Collect$$rtentry$$0000000B) for .ARM.Collect$$rtentry$$0000000B
    rtentry2.o(.ARM.exidx) refers to rtentry2.o(.ARM.Collect$$rtentry$$0000000D) for .ARM.Collect$$rtentry$$0000000D
    rtentry4.o(.ARM.Collect$$rtentry$$00000004) refers to sys_stackheap_outer.o(.text) for __user_setup_stackheap
    rtentry4.o(.ARM.exidx) refers to rtentry4.o(.ARM.Collect$$rtentry$$00000004) for .ARM.Collect$$rtentry$$00000004
    rt_div0.o(.text) refers to defsig_fpe_outer.o(.text) for __rt_SIGFPE
    sys_stackheap_outer.o(.text) refers to libspace.o(.text) for __user_perproc_libspace
    sys_stackheap_outer.o(.text) refers to startup_hhd32f0xx_s.o(.text) for __user_initial_stackheap
    sys_stackheap_outer.o(__vectab_stack_and_reset_area) refers to tempstk.o(.text) for __temporary_stack_top
    sys_stackheap_outer.o(__vectab_stack_and_reset_area) refers to __main.o(!!!main) for __main
    exit.o(.text) refers to rtexit.o(.ARM.Collect$$rtexit$$00000000) for __rt_exit
    defsig_fpe_outer.o(.text) refers to defsig_fpe_inner.o(.text) for __rt_SIGFPE_inner
    defsig_fpe_outer.o(.text) refers to defsig_exit.o(.text) for __sig_exit
    defsig_fpe_formal.o(.text) refers to rt_raise.o(.text) for __rt_raise
    libinit.o(.ARM.Collect$$libinit$$00000000) refers (Special) to libinit2.o(.ARM.Collect$$libinit$$0000002C) for __rt_lib_init_alloca_1
    libinit.o(.ARM.Collect$$libinit$$00000000) refers (Special) to libinit2.o(.ARM.Collect$$libinit$$0000002A) for __rt_lib_init_argv_1
    libinit.o(.ARM.Collect$$libinit$$00000000) refers (Special) to libinit2.o(.ARM.Collect$$libinit$$00000019) for __rt_lib_init_atexit_1
    libinit.o(.ARM.Collect$$libinit$$00000000) refers (Special) to libinit2.o(.ARM.Collect$$libinit$$0000001F) for __rt_lib_init_clock_1
    libinit.o(.ARM.Collect$$libinit$$00000000) refers (Special) to libinit2.o(.ARM.Collect$$libinit$$00000030) for __rt_lib_init_cpp_1
    libinit.o(.ARM.Collect$$libinit$$00000000) refers (Special) to libinit2.o(.ARM.Collect$$libinit$$0000002E) for __rt_lib_init_exceptions_1
    libinit.o(.ARM.Collect$$libinit$$00000000) refers (Special) to libinit2.o(.ARM.Collect$$libinit$$00000001) for __rt_lib_init_fp_1
    libinit.o(.ARM.Collect$$libinit$$00000000) refers (Special) to libinit2.o(.ARM.Collect$$libinit$$0000001D) for __rt_lib_init_fp_trap_1
    libinit.o(.ARM.Collect$$libinit$$00000000) refers (Special) to libinit2.o(.ARM.Collect$$libinit$$00000021) for __rt_lib_init_getenv_1
    libinit.o(.ARM.Collect$$libinit$$00000000) refers (Special) to libinit2.o(.ARM.Collect$$libinit$$00000008) for __rt_lib_init_heap_1
    libinit.o(.ARM.Collect$$libinit$$00000000) refers (Special) to libinit2.o(.ARM.Collect$$libinit$$0000000F) for __rt_lib_init_lc_collate_1
    libinit.o(.ARM.Collect$$libinit$$00000000) refers (Special) to libinit2.o(.ARM.Collect$$libinit$$00000011) for __rt_lib_init_lc_ctype_1
    libinit.o(.ARM.Collect$$libinit$$00000000) refers (Special) to libinit2.o(.ARM.Collect$$libinit$$00000013) for __rt_lib_init_lc_monetary_1
    libinit.o(.ARM.Collect$$libinit$$00000000) refers (Special) to libinit2.o(.ARM.Collect$$libinit$$00000015) for __rt_lib_init_lc_numeric_1
    libinit.o(.ARM.Collect$$libinit$$00000000) refers (Special) to libinit2.o(.ARM.Collect$$libinit$$00000017) for __rt_lib_init_lc_time_1
    libinit.o(.ARM.Collect$$libinit$$00000000) refers (Special) to libinit2.o(.ARM.Collect$$libinit$$0000000C) for __rt_lib_init_rand_1
    libinit.o(.ARM.Collect$$libinit$$00000000) refers (Special) to libinit2.o(.ARM.Collect$$libinit$$00000031) for __rt_lib_init_return
    libinit.o(.ARM.Collect$$libinit$$00000000) refers (Special) to libinit2.o(.ARM.Collect$$libinit$$0000001B) for __rt_lib_init_signal_1
    libinit.o(.ARM.Collect$$libinit$$00000000) refers (Special) to libinit2.o(.ARM.Collect$$libinit$$00000023) for __rt_lib_init_stdio_1
    libinit.o(.ARM.Collect$$libinit$$00000000) refers (Special) to libinit2.o(.ARM.Collect$$libinit$$0000000A) for __rt_lib_init_user_alloc_1
    libspace.o(.text) refers to libspace.o(.bss) for __libspace_start
    rtexit.o(.ARM.Collect$$rtexit$$00000000) refers (Special) to rtexit2.o(.ARM.Collect$$rtexit$$00000004) for __rt_exit_exit
    rtexit.o(.ARM.Collect$$rtexit$$00000000) refers (Special) to rtexit2.o(.ARM.Collect$$rtexit$$00000003) for __rt_exit_ls
    rtexit.o(.ARM.Collect$$rtexit$$00000000) refers (Special) to rtexit2.o(.ARM.Collect$$rtexit$$00000002) for __rt_exit_prels_1
    rtexit.o(.ARM.exidx) refers (Special) to rtexit2.o(.ARM.Collect$$rtexit$$00000004) for __rt_exit_exit
    rtexit.o(.ARM.exidx) refers (Special) to rtexit2.o(.ARM.Collect$$rtexit$$00000003) for __rt_exit_ls
    rtexit.o(.ARM.exidx) refers (Special) to rtexit2.o(.ARM.Collect$$rtexit$$00000002) for __rt_exit_prels_1
    rtexit.o(.ARM.exidx) refers to rtexit.o(.ARM.Collect$$rtexit$$00000000) for .ARM.Collect$$rtexit$$00000000
    rt_raise.o(.text) refers to __raise.o(.text) for __raise
    rt_raise.o(.text) refers to sys_exit.o(.text) for _sys_exit
    defsig_exit.o(.text) refers to sys_exit.o(.text) for _sys_exit
    defsig_fpe_inner.o(.text) refers to defsig_general.o(.text) for __default_signal_display
    libinit2.o(.ARM.Collect$$libinit$$0000000E) refers to libinit2.o(.ARM.Collect$$libinit$$0000000D) for .ARM.Collect$$libinit$$0000000D
    libinit2.o(.ARM.Collect$$libinit$$00000010) refers to libinit2.o(.ARM.Collect$$libinit$$0000000D) for .ARM.Collect$$libinit$$0000000D
    libinit2.o(.ARM.Collect$$libinit$$00000012) refers to libinit2.o(.ARM.Collect$$libinit$$0000000D) for .ARM.Collect$$libinit$$0000000D
    libinit2.o(.ARM.Collect$$libinit$$00000014) refers to libinit2.o(.ARM.Collect$$libinit$$0000000D) for .ARM.Collect$$libinit$$0000000D
    libinit2.o(.ARM.Collect$$libinit$$00000016) refers to libinit2.o(.ARM.Collect$$libinit$$0000000D) for .ARM.Collect$$libinit$$0000000D
    libinit2.o(.ARM.Collect$$libinit$$00000024) refers to argv_veneer.o(.text) for __ARM_argv_veneer
    libinit2.o(.ARM.Collect$$libinit$$00000025) refers to argv_veneer.o(.text) for __ARM_argv_veneer
    sys_exit.o(.text) refers (Special) to use_no_semi.o(.text) for __I$use$semihosting
    sys_exit.o(.text) refers (Special) to indicate_semi.o(.text) for __semihosting_library_function
    rtexit2.o(.ARM.Collect$$rtexit$$00000003) refers to libshutdown.o(.ARM.Collect$$libshutdown$$00000000) for __rt_lib_shutdown
    rtexit2.o(.ARM.Collect$$rtexit$$00000004) refers to sys_exit.o(.text) for _sys_exit
    rtexit2.o(.ARM.exidx) refers to rtexit2.o(.ARM.Collect$$rtexit$$00000001) for .ARM.Collect$$rtexit$$00000001
    rtexit2.o(.ARM.exidx) refers to rtexit2.o(.ARM.Collect$$rtexit$$00000003) for .ARM.Collect$$rtexit$$00000003
    rtexit2.o(.ARM.exidx) refers to rtexit2.o(.ARM.Collect$$rtexit$$00000004) for .ARM.Collect$$rtexit$$00000004
    __raise.o(.text) refers to defsig.o(CL$$defsig) for __default_signal_handler
    defsig_general.o(.text) refers to sys_wrch.o(.text) for _ttywrch
    sys_wrch.o(.text) refers (Special) to use_no_semi.o(.text) for __I$use$semihosting
    sys_wrch.o(.text) refers (Special) to indicate_semi.o(.text) for __semihosting_library_function
    defsig.o(CL$$defsig) refers to defsig_fpe_inner.o(.text) for __rt_SIGFPE_inner
    defsig.o(CL$$defsig) refers to defsig_rtmem_inner.o(.text) for __rt_SIGRTMEM_inner
    _get_argv_nomalloc.o(.text) refers (Special) to hrguard.o(.text) for __heap_region$guard
    _get_argv_nomalloc.o(.text) refers to defsig_rtmem_outer.o(.text) for __rt_SIGRTMEM
    _get_argv_nomalloc.o(.text) refers to sys_command.o(.text) for _sys_command_string
    libshutdown.o(.ARM.Collect$$libshutdown$$00000000) refers (Special) to libshutdown2.o(.ARM.Collect$$libshutdown$$00000006) for __rt_lib_shutdown_fp_trap_1
    libshutdown.o(.ARM.Collect$$libshutdown$$00000000) refers (Special) to libshutdown2.o(.ARM.Collect$$libshutdown$$0000000E) for __rt_lib_shutdown_heap_1
    libshutdown.o(.ARM.Collect$$libshutdown$$00000000) refers (Special) to libshutdown2.o(.ARM.Collect$$libshutdown$$0000000F) for __rt_lib_shutdown_return
    libshutdown.o(.ARM.Collect$$libshutdown$$00000000) refers (Special) to libshutdown2.o(.ARM.Collect$$libshutdown$$00000009) for __rt_lib_shutdown_signal_1
    libshutdown.o(.ARM.Collect$$libshutdown$$00000000) refers (Special) to libshutdown2.o(.ARM.Collect$$libshutdown$$00000003) for __rt_lib_shutdown_stdio_1
    libshutdown.o(.ARM.Collect$$libshutdown$$00000000) refers (Special) to libshutdown2.o(.ARM.Collect$$libshutdown$$0000000B) for __rt_lib_shutdown_user_alloc_1
    sys_command.o(.text) refers (Special) to use_no_semi.o(.text) for __I$use$semihosting
    sys_command.o(.text) refers (Special) to indicate_semi.o(.text) for __semihosting_library_function
    defsig_abrt_inner.o(.text) refers to defsig_general.o(.text) for __default_signal_display
    defsig_rtred_inner.o(.text) refers to defsig_general.o(.text) for __default_signal_display
    defsig_rtmem_inner.o(.text) refers to defsig_general.o(.text) for __default_signal_display
    defsig_rtmem_outer.o(.text) refers to defsig_rtmem_inner.o(.text) for __rt_SIGRTMEM_inner
    defsig_rtmem_outer.o(.text) refers to defsig_exit.o(.text) for __sig_exit
    defsig_rtmem_formal.o(.text) refers to rt_raise.o(.text) for __rt_raise
    defsig_stak_inner.o(.text) refers to defsig_general.o(.text) for __default_signal_display
    defsig_pvfn_inner.o(.text) refers to defsig_general.o(.text) for __default_signal_display
    defsig_cppl_inner.o(.text) refers to defsig_general.o(.text) for __default_signal_display
    defsig_segv_inner.o(.text) refers to defsig_general.o(.text) for __default_signal_display
    defsig_other.o(.text) refers to defsig_general.o(.text) for __default_signal_display


==============================================================================

Removing Unused input sections from the image.

    Removing hhd_sys.o(.rev16_text), (4 bytes).
    Removing hhd_sys.o(.revsh_text), (4 bytes).
    Removing hhd_uart.o(.rev16_text), (4 bytes).
    Removing hhd_uart.o(.revsh_text), (4 bytes).
    Removing hhd_iic.o(.rev16_text), (4 bytes).
    Removing hhd_iic.o(.revsh_text), (4 bytes).
    Removing system_hhd32f0xx.o(.rev16_text), (4 bytes).
    Removing system_hhd32f0xx.o(.revsh_text), (4 bytes).
    Removing main.o(.rev16_text), (4 bytes).
    Removing main.o(.revsh_text), (4 bytes).
    Removing main.o(.data), (41 bytes).
    Removing lm75a.o(.rev16_text), (4 bytes).
    Removing lm75a.o(.revsh_text), (4 bytes).
    Removing lm75a.o(.text), (22 bytes).
    Removing lm75a.o(.data), (41 bytes).
    Removing sd2405alpi.o(.rev16_text), (4 bytes).
    Removing sd2405alpi.o(.revsh_text), (4 bytes).
    Removing sd2405alpi.o(.text), (76 bytes).
    Removing sd2405alpi.o(.data), (41 bytes).
    Removing at24c02.o(.rev16_text), (4 bytes).
    Removing at24c02.o(.revsh_text), (4 bytes).
    Removing at24c02.o(.data), (41 bytes).

22 unused section(s) (total 326 bytes) removed from the image.

==============================================================================

Image Symbol Table

    Local Symbols

    Symbol Name                              Value     Ov Type        Size  Object(Section)

    RESET                                    0x00000000   Section      192  startup_hhd32f0xx_s.o(RESET)
    ../clib/angel/boardlib.s                 0x00000000   Number         0  boardinit2.o ABSOLUTE
    ../clib/angel/boardlib.s                 0x00000000   Number         0  boardinit3.o ABSOLUTE
    ../clib/angel/boardlib.s                 0x00000000   Number         0  boardshut.o ABSOLUTE
    ../clib/angel/boardlib.s                 0x00000000   Number         0  boardinit1.o ABSOLUTE
    ../clib/angel/handlers.s                 0x00000000   Number         0  __scatter_zi.o ABSOLUTE
    ../clib/angel/handlers.s                 0x00000000   Number         0  __scatter_copy.o ABSOLUTE
    ../clib/angel/kernel.s                   0x00000000   Number         0  rtexit.o ABSOLUTE
    ../clib/angel/kernel.s                   0x00000000   Number         0  rtentry4.o ABSOLUTE
    ../clib/angel/kernel.s                   0x00000000   Number         0  rtexit2.o ABSOLUTE
    ../clib/angel/kernel.s                   0x00000000   Number         0  rtentry2.o ABSOLUTE
    ../clib/angel/kernel.s                   0x00000000   Number         0  rtentry.o ABSOLUTE
    ../clib/angel/rt.s                       0x00000000   Number         0  rt_raise.o ABSOLUTE
    ../clib/angel/rt.s                       0x00000000   Number         0  rt_div0.o ABSOLUTE
    ../clib/angel/rt.s                       0x00000000   Number         0  aeabi_idiv0_sigfpe.o ABSOLUTE
    ../clib/angel/rt.s                       0x00000000   Number         0  aeabi_idiv0.o ABSOLUTE
    ../clib/angel/scatterp.s                 0x00000000   Number         0  __scatter.o ABSOLUTE
    ../clib/angel/startup.s                  0x00000000   Number         0  __main.o ABSOLUTE
    ../clib/angel/sys.s                      0x00000000   Number         0  use_no_semi.o ABSOLUTE
    ../clib/angel/sys.s                      0x00000000   Number         0  indicate_semi.o ABSOLUTE
    ../clib/angel/sys.s                      0x00000000   Number         0  tempstk.o ABSOLUTE
    ../clib/angel/sys.s                      0x00000000   Number         0  sys_stackheap_outer.o ABSOLUTE
    ../clib/angel/sys.s                      0x00000000   Number         0  libspace.o ABSOLUTE
    ../clib/angel/sysapp.c                   0x00000000   Number         0  sys_exit.o ABSOLUTE
    ../clib/angel/sysapp.c                   0x00000000   Number         0  sys_command.o ABSOLUTE
    ../clib/angel/sysapp.c                   0x00000000   Number         0  sys_wrch.o ABSOLUTE
    ../clib/armsys.c                         0x00000000   Number         0  _get_argv_nomalloc.o ABSOLUTE
    ../clib/armsys.c                         0x00000000   Number         0  argv_veneer.o ABSOLUTE
    ../clib/armsys.c                         0x00000000   Number         0  no_argv.o ABSOLUTE
    ../clib/division.s                       0x00000000   Number         0  aeabi_sdiv_div0.o ABSOLUTE
    ../clib/division.s                       0x00000000   Number         0  aeabi_sdiv.o ABSOLUTE
    ../clib/heapalloc.c                      0x00000000   Number         0  hrguard.o ABSOLUTE
    ../clib/heapaux.c                        0x00000000   Number         0  heapauxi.o ABSOLUTE
    ../clib/libinit.s                        0x00000000   Number         0  libshutdown2.o ABSOLUTE
    ../clib/libinit.s                        0x00000000   Number         0  libshutdown.o ABSOLUTE
    ../clib/libinit.s                        0x00000000   Number         0  libinit2.o ABSOLUTE
    ../clib/libinit.s                        0x00000000   Number         0  libinit.o ABSOLUTE
    ../clib/signal.c                         0x00000000   Number         0  defsig_stak_inner.o ABSOLUTE
    ../clib/signal.c                         0x00000000   Number         0  defsig_rtmem_formal.o ABSOLUTE
    ../clib/signal.c                         0x00000000   Number         0  defsig_rtmem_outer.o ABSOLUTE
    ../clib/signal.c                         0x00000000   Number         0  defsig_pvfn_inner.o ABSOLUTE
    ../clib/signal.c                         0x00000000   Number         0  defsig_cppl_inner.o ABSOLUTE
    ../clib/signal.c                         0x00000000   Number         0  defsig_fpe_inner.o ABSOLUTE
    ../clib/signal.c                         0x00000000   Number         0  defsig_exit.o ABSOLUTE
    ../clib/signal.c                         0x00000000   Number         0  defsig_segv_inner.o ABSOLUTE
    ../clib/signal.c                         0x00000000   Number         0  defsig_other.o ABSOLUTE
    ../clib/signal.c                         0x00000000   Number         0  defsig_fpe_outer.o ABSOLUTE
    ../clib/signal.c                         0x00000000   Number         0  defsig_fpe_formal.o ABSOLUTE
    ../clib/signal.c                         0x00000000   Number         0  __raise.o ABSOLUTE
    ../clib/signal.c                         0x00000000   Number         0  defsig_abrt_inner.o ABSOLUTE
    ../clib/signal.c                         0x00000000   Number         0  defsig_rtred_inner.o ABSOLUTE
    ../clib/signal.c                         0x00000000   Number         0  defsig_general.o ABSOLUTE
    ../clib/signal.c                         0x00000000   Number         0  defsig_rtmem_inner.o ABSOLUTE
    ../clib/signal.s                         0x00000000   Number         0  defsig.o ABSOLUTE
    ../clib/stdlib.c                         0x00000000   Number         0  exit.o ABSOLUTE
    ../fplib/cfplib/fpinit.c                 0x00000000   Number         0  fpinit.o ABSOLUTE
    ..\..\HHD32F0xx_library\Core\CM0\CoreSupport\core_cm0.c 0x00000000   Number         0  core_cm0.o ABSOLUTE
    ..\..\HHD32F0xx_library\Core\CM0\DeviceSupport\HHD32F0xx\startup\arm\startup_hhd32F0xx_s.s 0x00000000   Number         0  startup_hhd32f0xx_s.o ABSOLUTE
    ..\..\HHD32F0xx_library\Core\CM0\DeviceSupport\HHD32F0xx\system_hhd32f0xx.c 0x00000000   Number         0  system_hhd32f0xx.o ABSOLUTE
    ..\..\HHD32F0xx_library\Drivers\source\hhd_iic.c 0x00000000   Number         0  hhd_iic.o ABSOLUTE
    ..\..\HHD32F0xx_library\Drivers\source\hhd_sys.c 0x00000000   Number         0  hhd_sys.o ABSOLUTE
    ..\..\HHD32F0xx_library\Drivers\source\hhd_uart.c 0x00000000   Number         0  hhd_uart.o ABSOLUTE
    ..\\..\\HHD32F0xx_library\\Core\\CM0\\DeviceSupport\\HHD32F0xx\\system_hhd32f0xx.c 0x00000000   Number         0  system_hhd32f0xx.o ABSOLUTE
    ..\\..\\HHD32F0xx_library\\Drivers\\source\\hhd_iic.c 0x00000000   Number         0  hhd_iic.o ABSOLUTE
    ..\\..\\HHD32F0xx_library\\Drivers\\source\\hhd_sys.c 0x00000000   Number         0  hhd_sys.o ABSOLUTE
    ..\\..\\HHD32F0xx_library\\Drivers\\source\\hhd_uart.c 0x00000000   Number         0  hhd_uart.o ABSOLUTE
    dc.s                                     0x00000000   Number         0  dc.o ABSOLUTE
    myapp\\src\\AT24C02.c                    0x00000000   Number         0  at24c02.o ABSOLUTE
    myapp\\src\\LM75A.c                      0x00000000   Number         0  lm75a.o ABSOLUTE
    myapp\\src\\SD2405ALPI.c                 0x00000000   Number         0  sd2405alpi.o ABSOLUTE
    myapp\\src\\main.c                       0x00000000   Number         0  main.o ABSOLUTE
    myapp\src\AT24C02.c                      0x00000000   Number         0  at24c02.o ABSOLUTE
    myapp\src\LM75A.c                        0x00000000   Number         0  lm75a.o ABSOLUTE
    myapp\src\SD2405ALPI.c                   0x00000000   Number         0  sd2405alpi.o ABSOLUTE
    myapp\src\main.c                         0x00000000   Number         0  main.o ABSOLUTE
    !!!main                                  0x000000c0   Section        8  __main.o(!!!main)
    !!!scatter                               0x000000c8   Section       60  __scatter.o(!!!scatter)
    !!handler_copy                           0x00000104   Section       26  __scatter_copy.o(!!handler_copy)
    !!handler_zi                             0x00000120   Section       28  __scatter_zi.o(!!handler_zi)
    .ARM.Collect$$libinit$$00000000          0x0000013c   Section        2  libinit.o(.ARM.Collect$$libinit$$00000000)
    .ARM.Collect$$libinit$$00000001          0x0000013e   Section        4  libinit2.o(.ARM.Collect$$libinit$$00000001)
    .ARM.Collect$$libinit$$00000008          0x00000142   Section        0  libinit2.o(.ARM.Collect$$libinit$$00000008)
    .ARM.Collect$$libinit$$0000000A          0x00000142   Section        0  libinit2.o(.ARM.Collect$$libinit$$0000000A)
    .ARM.Collect$$libinit$$0000000C          0x00000142   Section        0  libinit2.o(.ARM.Collect$$libinit$$0000000C)
    .ARM.Collect$$libinit$$0000000F          0x00000142   Section        0  libinit2.o(.ARM.Collect$$libinit$$0000000F)
    .ARM.Collect$$libinit$$00000011          0x00000142   Section        0  libinit2.o(.ARM.Collect$$libinit$$00000011)
    .ARM.Collect$$libinit$$00000013          0x00000142   Section        0  libinit2.o(.ARM.Collect$$libinit$$00000013)
    .ARM.Collect$$libinit$$00000015          0x00000142   Section        0  libinit2.o(.ARM.Collect$$libinit$$00000015)
    .ARM.Collect$$libinit$$00000017          0x00000142   Section        0  libinit2.o(.ARM.Collect$$libinit$$00000017)
    .ARM.Collect$$libinit$$00000019          0x00000142   Section        0  libinit2.o(.ARM.Collect$$libinit$$00000019)
    .ARM.Collect$$libinit$$0000001B          0x00000142   Section        0  libinit2.o(.ARM.Collect$$libinit$$0000001B)
    .ARM.Collect$$libinit$$0000001D          0x00000142   Section        0  libinit2.o(.ARM.Collect$$libinit$$0000001D)
    .ARM.Collect$$libinit$$0000001F          0x00000142   Section        0  libinit2.o(.ARM.Collect$$libinit$$0000001F)
    .ARM.Collect$$libinit$$00000021          0x00000142   Section        0  libinit2.o(.ARM.Collect$$libinit$$00000021)
    .ARM.Collect$$libinit$$00000023          0x00000142   Section        0  libinit2.o(.ARM.Collect$$libinit$$00000023)
    .ARM.Collect$$libinit$$0000002A          0x00000142   Section        0  libinit2.o(.ARM.Collect$$libinit$$0000002A)
    .ARM.Collect$$libinit$$0000002C          0x00000142   Section        0  libinit2.o(.ARM.Collect$$libinit$$0000002C)
    .ARM.Collect$$libinit$$0000002E          0x00000142   Section        0  libinit2.o(.ARM.Collect$$libinit$$0000002E)
    .ARM.Collect$$libinit$$00000030          0x00000142   Section        0  libinit2.o(.ARM.Collect$$libinit$$00000030)
    .ARM.Collect$$libinit$$00000031          0x00000142   Section        2  libinit2.o(.ARM.Collect$$libinit$$00000031)
    .ARM.Collect$$libshutdown$$00000000      0x00000144   Section        2  libshutdown.o(.ARM.Collect$$libshutdown$$00000000)
    .ARM.Collect$$libshutdown$$00000003      0x00000146   Section        0  libshutdown2.o(.ARM.Collect$$libshutdown$$00000003)
    .ARM.Collect$$libshutdown$$00000006      0x00000146   Section        0  libshutdown2.o(.ARM.Collect$$libshutdown$$00000006)
    .ARM.Collect$$libshutdown$$00000009      0x00000146   Section        0  libshutdown2.o(.ARM.Collect$$libshutdown$$00000009)
    .ARM.Collect$$libshutdown$$0000000B      0x00000146   Section        0  libshutdown2.o(.ARM.Collect$$libshutdown$$0000000B)
    .ARM.Collect$$libshutdown$$0000000E      0x00000146   Section        0  libshutdown2.o(.ARM.Collect$$libshutdown$$0000000E)
    .ARM.Collect$$libshutdown$$0000000F      0x00000146   Section        2  libshutdown2.o(.ARM.Collect$$libshutdown$$0000000F)
    .ARM.Collect$$rtentry$$00000000          0x00000148   Section        0  rtentry.o(.ARM.Collect$$rtentry$$00000000)
    .ARM.Collect$$rtentry$$00000002          0x00000148   Section        0  rtentry2.o(.ARM.Collect$$rtentry$$00000002)
    .ARM.Collect$$rtentry$$00000004          0x00000148   Section        6  rtentry4.o(.ARM.Collect$$rtentry$$00000004)
    .ARM.Collect$$rtentry$$00000009          0x0000014e   Section        0  rtentry2.o(.ARM.Collect$$rtentry$$00000009)
    .ARM.Collect$$rtentry$$0000000A          0x0000014e   Section        4  rtentry2.o(.ARM.Collect$$rtentry$$0000000A)
    .ARM.Collect$$rtentry$$0000000C          0x00000152   Section        0  rtentry2.o(.ARM.Collect$$rtentry$$0000000C)
    .ARM.Collect$$rtentry$$0000000D          0x00000152   Section        8  rtentry2.o(.ARM.Collect$$rtentry$$0000000D)
    .ARM.Collect$$rtexit$$00000000           0x0000015a   Section        2  rtexit.o(.ARM.Collect$$rtexit$$00000000)
    .ARM.Collect$$rtexit$$00000002           0x0000015c   Section        0  rtexit2.o(.ARM.Collect$$rtexit$$00000002)
    .ARM.Collect$$rtexit$$00000003           0x0000015c   Section        4  rtexit2.o(.ARM.Collect$$rtexit$$00000003)
    .ARM.Collect$$rtexit$$00000004           0x00000160   Section        6  rtexit2.o(.ARM.Collect$$rtexit$$00000004)
    .text                                    0x00000168   Section        0  hhd_sys.o(.text)
    .text                                    0x00000568   Section        0  hhd_uart.o(.text)
    NVIC_DisableIRQ                          0x000007fb   Thumb Code    14  hhd_uart.o(.text)
    .text                                    0x0000081c   Section        0  hhd_iic.o(.text)
    .text                                    0x00000ca8   Section        0  system_hhd32f0xx.o(.text)
    .text                                    0x00000d18   Section       48  startup_hhd32f0xx_s.o(.text)
    .text                                    0x00000d48   Section        0  main.o(.text)
    .text                                    0x00000d9c   Section        0  at24c02.o(.text)
    .text                                    0x00000dbc   Section      346  aeabi_sdiv.o(.text)
    .text                                    0x00000f16   Section        0  heapauxi.o(.text)
    .text                                    0x00000f1c   Section       62  sys_stackheap_outer.o(.text)
    .text                                    0x00000f5a   Section        0  exit.o(.text)
    .text                                    0x00000f68   Section        8  libspace.o(.text)
    .text                                    0x00000f70   Section        0  sys_exit.o(.text)
    .text                                    0x00000f7c   Section        2  use_no_semi.o(.text)
    .text                                    0x00000f7e   Section        0  indicate_semi.o(.text)
    i.__ARM_common_switch8                   0x00000f7e   Section        0  hhd_sys.o(i.__ARM_common_switch8)
    .data                                    0x10000000   Section       41  hhd_iic.o(.data)
    IICMasterState                           0x10000000   Data           1  hhd_iic.o(.data)
    RdIndex                                  0x10000004   Data           4  hhd_iic.o(.data)
    WrIndex                                  0x10000008   Data           4  hhd_iic.o(.data)
    Restart                                  0x1000000c   Data           4  hhd_iic.o(.data)
    IICMasterBuffer                          0x10000010   Data           8  hhd_iic.o(.data)
    IICSlaveBuffer                           0x10000018   Data           8  hhd_iic.o(.data)
    IICReadLength                            0x10000020   Data           4  hhd_iic.o(.data)
    IICWriteLength                           0x10000024   Data           4  hhd_iic.o(.data)
    Re_Start                                 0x10000028   Data           1  hhd_iic.o(.data)
    .data                                    0x1000002c   Section        8  system_hhd32f0xx.o(.data)
    .bss                                     0x10000034   Section       96  libspace.o(.bss)
    HEAP                                     0x10000098   Section      256  startup_hhd32f0xx_s.o(HEAP)
    Heap_Mem                                 0x10000098   Data         256  startup_hhd32f0xx_s.o(HEAP)
    STACK                                    0x10000198   Section      512  startup_hhd32f0xx_s.o(STACK)
    Stack_Mem                                0x10000198   Data         512  startup_hhd32f0xx_s.o(STACK)
    __initial_sp                             0x10000398   Data           0  startup_hhd32f0xx_s.o(STACK)

    Global Symbols

    Symbol Name                              Value     Ov Type        Size  Object(Section)

    BuildAttributes$$THM_ISAv3M$S$PE$A:L22$X:L11$S22$IEEE1$IW$USESV6$~STKCKD$USESV7$~SHL$OSPACE$ROPI$EBA8$UX$STANDARDLIB$REQ8$PRES8$EABIv2 0x00000000   Number         0  anon$$obj.o ABSOLUTE
    __ARM_use_no_argv                        0x00000000   Number         0  main.o ABSOLUTE
    __Vectors                                0x00000000   Data           4  startup_hhd32f0xx_s.o(RESET)
    __ARM_exceptions_init                     - Undefined Weak Reference
    __alloca_initialize                       - Undefined Weak Reference
    __cpp_initialize__aeabi_                  - Undefined Weak Reference
    __cxa_finalize                            - Undefined Weak Reference
    __rt_locale                               - Undefined Weak Reference
    __sigvec_lookup                           - Undefined Weak Reference
    _atexit_init                              - Undefined Weak Reference
    _call_atexit_fns                          - Undefined Weak Reference
    _clock_init                               - Undefined Weak Reference
    _fp_trap_init                             - Undefined Weak Reference
    _fp_trap_shutdown                         - Undefined Weak Reference
    _get_lc_collate                           - Undefined Weak Reference
    _get_lc_ctype                             - Undefined Weak Reference
    _get_lc_monetary                          - Undefined Weak Reference
    _get_lc_numeric                           - Undefined Weak Reference
    _get_lc_time                              - Undefined Weak Reference
    _getenv_init                              - Undefined Weak Reference
    _handle_redirection                       - Undefined Weak Reference
    _init_alloc                               - Undefined Weak Reference
    _init_user_alloc                          - Undefined Weak Reference
    _initio                                   - Undefined Weak Reference
    _rand_init                                - Undefined Weak Reference
    _signal_finish                            - Undefined Weak Reference
    _signal_init                              - Undefined Weak Reference
    _terminate_alloc                          - Undefined Weak Reference
    _terminate_user_alloc                     - Undefined Weak Reference
    _terminateio                              - Undefined Weak Reference
    __Vectors_End                            0x000000c0   Data           0  startup_hhd32f0xx_s.o(RESET)
    __Vectors_Size                           0x000000c0   Number         0  startup_hhd32f0xx_s.o ABSOLUTE
    __main                                   0x000000c1   Thumb Code     8  __main.o(!!!main)
    __scatterload                            0x000000c9   Thumb Code     0  __scatter.o(!!!scatter)
    __scatterload_rt2                        0x000000c9   Thumb Code    52  __scatter.o(!!!scatter)
    __scatterload_rt2_thumb_only             0x000000c9   Thumb Code     0  __scatter.o(!!!scatter)
    __scatterload_null                       0x000000d9   Thumb Code     0  __scatter.o(!!!scatter)
    __scatterload_copy                       0x00000105   Thumb Code    26  __scatter_copy.o(!!handler_copy)
    __scatterload_zeroinit                   0x00000121   Thumb Code    28  __scatter_zi.o(!!handler_zi)
    __rt_lib_init                            0x0000013d   Thumb Code     0  libinit.o(.ARM.Collect$$libinit$$00000000)
    __rt_lib_init_fp_1                       0x0000013f   Thumb Code     0  libinit2.o(.ARM.Collect$$libinit$$00000001)
    __rt_lib_init_alloca_1                   0x00000143   Thumb Code     0  libinit2.o(.ARM.Collect$$libinit$$0000002C)
    __rt_lib_init_argv_1                     0x00000143   Thumb Code     0  libinit2.o(.ARM.Collect$$libinit$$0000002A)
    __rt_lib_init_atexit_1                   0x00000143   Thumb Code     0  libinit2.o(.ARM.Collect$$libinit$$00000019)
    __rt_lib_init_clock_1                    0x00000143   Thumb Code     0  libinit2.o(.ARM.Collect$$libinit$$0000001F)
    __rt_lib_init_cpp_1                      0x00000143   Thumb Code     0  libinit2.o(.ARM.Collect$$libinit$$00000030)
    __rt_lib_init_exceptions_1               0x00000143   Thumb Code     0  libinit2.o(.ARM.Collect$$libinit$$0000002E)
    __rt_lib_init_fp_trap_1                  0x00000143   Thumb Code     0  libinit2.o(.ARM.Collect$$libinit$$0000001D)
    __rt_lib_init_getenv_1                   0x00000143   Thumb Code     0  libinit2.o(.ARM.Collect$$libinit$$00000021)
    __rt_lib_init_heap_1                     0x00000143   Thumb Code     0  libinit2.o(.ARM.Collect$$libinit$$00000008)
    __rt_lib_init_lc_collate_1               0x00000143   Thumb Code     0  libinit2.o(.ARM.Collect$$libinit$$0000000F)
    __rt_lib_init_lc_ctype_1                 0x00000143   Thumb Code     0  libinit2.o(.ARM.Collect$$libinit$$00000011)
    __rt_lib_init_lc_monetary_1              0x00000143   Thumb Code     0  libinit2.o(.ARM.Collect$$libinit$$00000013)
    __rt_lib_init_lc_numeric_1               0x00000143   Thumb Code     0  libinit2.o(.ARM.Collect$$libinit$$00000015)
    __rt_lib_init_lc_time_1                  0x00000143   Thumb Code     0  libinit2.o(.ARM.Collect$$libinit$$00000017)
    __rt_lib_init_rand_1                     0x00000143   Thumb Code     0  libinit2.o(.ARM.Collect$$libinit$$0000000C)
    __rt_lib_init_return                     0x00000143   Thumb Code     0  libinit2.o(.ARM.Collect$$libinit$$00000031)
    __rt_lib_init_signal_1                   0x00000143   Thumb Code     0  libinit2.o(.ARM.Collect$$libinit$$0000001B)
    __rt_lib_init_stdio_1                    0x00000143   Thumb Code     0  libinit2.o(.ARM.Collect$$libinit$$00000023)
    __rt_lib_init_user_alloc_1               0x00000143   Thumb Code     0  libinit2.o(.ARM.Collect$$libinit$$0000000A)
    __rt_lib_shutdown                        0x00000145   Thumb Code     0  libshutdown.o(.ARM.Collect$$libshutdown$$00000000)
    __rt_lib_shutdown_fp_trap_1              0x00000147   Thumb Code     0  libshutdown2.o(.ARM.Collect$$libshutdown$$00000006)
    __rt_lib_shutdown_heap_1                 0x00000147   Thumb Code     0  libshutdown2.o(.ARM.Collect$$libshutdown$$0000000E)
    __rt_lib_shutdown_return                 0x00000147   Thumb Code     0  libshutdown2.o(.ARM.Collect$$libshutdown$$0000000F)
    __rt_lib_shutdown_signal_1               0x00000147   Thumb Code     0  libshutdown2.o(.ARM.Collect$$libshutdown$$00000009)
    __rt_lib_shutdown_stdio_1                0x00000147   Thumb Code     0  libshutdown2.o(.ARM.Collect$$libshutdown$$00000003)
    __rt_lib_shutdown_user_alloc_1           0x00000147   Thumb Code     0  libshutdown2.o(.ARM.Collect$$libshutdown$$0000000B)
    __rt_entry                               0x00000149   Thumb Code     0  rtentry.o(.ARM.Collect$$rtentry$$00000000)
    __rt_entry_presh_1                       0x00000149   Thumb Code     0  rtentry2.o(.ARM.Collect$$rtentry$$00000002)
    __rt_entry_sh                            0x00000149   Thumb Code     0  rtentry4.o(.ARM.Collect$$rtentry$$00000004)
    __rt_entry_li                            0x0000014f   Thumb Code     0  rtentry2.o(.ARM.Collect$$rtentry$$0000000A)
    __rt_entry_postsh_1                      0x0000014f   Thumb Code     0  rtentry2.o(.ARM.Collect$$rtentry$$00000009)
    __rt_entry_main                          0x00000153   Thumb Code     0  rtentry2.o(.ARM.Collect$$rtentry$$0000000D)
    __rt_entry_postli_1                      0x00000153   Thumb Code     0  rtentry2.o(.ARM.Collect$$rtentry$$0000000C)
    __rt_exit                                0x0000015b   Thumb Code     0  rtexit.o(.ARM.Collect$$rtexit$$00000000)
    __rt_exit_ls                             0x0000015d   Thumb Code     0  rtexit2.o(.ARM.Collect$$rtexit$$00000003)
    __rt_exit_prels_1                        0x0000015d   Thumb Code     0  rtexit2.o(.ARM.Collect$$rtexit$$00000002)
    __rt_exit_exit                           0x00000161   Thumb Code     0  rtexit2.o(.ARM.Collect$$rtexit$$00000004)
    SYS_SystemInitial                        0x00000169   Thumb Code    40  hhd_sys.o(.text)
    SYS_SelectMainClkSrc                     0x00000191   Thumb Code    80  hhd_sys.o(.text)
    SYS_SetAHBClkDivider                     0x000001e1   Thumb Code    30  hhd_sys.o(.text)
    SYS_SelectWDTClkSrc                      0x000001ff   Thumb Code    42  hhd_sys.o(.text)
    SYS_SelectClkOutSrc                      0x00000229   Thumb Code    92  hhd_sys.o(.text)
    SYS_SetClkOutDivider                     0x00000285   Thumb Code    22  hhd_sys.o(.text)
    SYS_EnableClkOut                         0x0000029b   Thumb Code     8  hhd_sys.o(.text)
    SYS_DisableClkOut                        0x000002a3   Thumb Code    26  hhd_sys.o(.text)
    SYS_SetIOFilter                          0x000002bd   Thumb Code    18  hhd_sys.o(.text)
    SYS_PowerDownAngIP                       0x000002cf   Thumb Code    16  hhd_sys.o(.text)
    SYS_PowerUpAngIP                         0x000002df   Thumb Code    16  hhd_sys.o(.text)
    SYS_EnablePhrClk                         0x000002ef   Thumb Code    16  hhd_sys.o(.text)
    SYS_DisablePhrClk                        0x000002ff   Thumb Code    16  hhd_sys.o(.text)
    SYS_ResetPhr                             0x0000030f   Thumb Code    20  hhd_sys.o(.text)
    SYS_ResetSystem                          0x00000323   Thumb Code    22  hhd_sys.o(.text)
    SYS_BODResetSystem                       0x00000339   Thumb Code    48  hhd_sys.o(.text)
    SYS_GetResetStatus                       0x00000369   Thumb Code     6  hhd_sys.o(.text)
    SYS_ClearResetStatus                     0x0000036f   Thumb Code     8  hhd_sys.o(.text)
    SYS_EnterSleep                           0x00000377   Thumb Code    28  hhd_sys.o(.text)
    SYS_SetDeepSleepWakeupPin                0x00000393   Thumb Code    46  hhd_sys.o(.text)
    SYS_ResetDeepSleepWakeupPin              0x000003c1   Thumb Code    10  hhd_sys.o(.text)
    SYS_EnterDeepSleep                       0x000003cb   Thumb Code   166  hhd_sys.o(.text)
    SYS_EnterPowerDown                       0x00000471   Thumb Code   106  hhd_sys.o(.text)
    SYS_IOConfig                             0x000004db   Thumb Code     4  hhd_sys.o(.text)
    SYS_IOSetPullup                          0x000004df   Thumb Code    20  hhd_sys.o(.text)
    SYS_IOSetPulldown                        0x000004f3   Thumb Code    20  hhd_sys.o(.text)
    SYS_IOSwitchtoAng                        0x00000507   Thumb Code    12  hhd_sys.o(.text)
    SYS_IOSwitchtoDigit                      0x00000513   Thumb Code    14  hhd_sys.o(.text)
    SYS_IOEnableFilter                       0x00000521   Thumb Code    14  hhd_sys.o(.text)
    SYS_IODisableFilter                      0x0000052f   Thumb Code    12  hhd_sys.o(.text)
    UART_Open                                0x00000569   Thumb Code   284  hhd_uart.o(.text)
    UART_ClearIntFlag                        0x00000685   Thumb Code    10  hhd_uart.o(.text)
    UART_DisableInt                          0x0000068f   Thumb Code    10  hhd_uart.o(.text)
    UART_Close                               0x00000699   Thumb Code    74  hhd_uart.o(.text)
    UART_ByteRead                            0x000006e3   Thumb Code    22  hhd_uart.o(.text)
    UART_Read                                0x000006f9   Thumb Code    38  hhd_uart.o(.text)
    UART_ByteWrite                           0x0000071f   Thumb Code    30  hhd_uart.o(.text)
    UART_Write                               0x0000073d   Thumb Code    48  hhd_uart.o(.text)
    UART_Send                                0x0000076d   Thumb Code    38  hhd_uart.o(.text)
    UART_PutString                           0x00000793   Thumb Code    26  hhd_uart.o(.text)
    UART_PutHex                              0x000007ad   Thumb Code    56  hhd_uart.o(.text)
    UART_EnableInt                           0x000007e5   Thumb Code     8  hhd_uart.o(.text)
    UART_GetStatus                           0x000007ed   Thumb Code     8  hhd_uart.o(.text)
    UART_ClearFIFO                           0x000007f5   Thumb Code     6  hhd_uart.o(.text)
    IIC_Init                                 0x0000081d   Thumb Code   196  hhd_iic.o(.text)
    IIC_GetIICStatus                         0x000008e1   Thumb Code    10  hhd_iic.o(.text)
    IIC_ReadFlag                             0x000008eb   Thumb Code    12  hhd_iic.o(.text)
    IIC_SetFlag                              0x000008f7   Thumb Code     8  hhd_iic.o(.text)
    IIC_ClearFlag                            0x000008ff   Thumb Code     8  hhd_iic.o(.text)
    IIC_SendByte                             0x00000907   Thumb Code     8  hhd_iic.o(.text)
    IIC_GetByte                              0x0000090f   Thumb Code    10  hhd_iic.o(.text)
    IIC_IRQHandler                           0x00000919   Thumb Code   526  hhd_iic.o(.text)
    IIC_WriteByte                            0x00000b27   Thumb Code    68  hhd_iic.o(.text)
    IIC_WriteArray                           0x00000b6b   Thumb Code    88  hhd_iic.o(.text)
    IIC_ReadByte                             0x00000bc3   Thumb Code   118  hhd_iic.o(.text)
    IIC_ReadArray                            0x00000c39   Thumb Code    86  hhd_iic.o(.text)
    SystemCoreClockUpdate                    0x00000ca9   Thumb Code    90  system_hhd32f0xx.o(.text)
    SystemInit                               0x00000d03   Thumb Code     2  system_hhd32f0xx.o(.text)
    Reset_Handler                            0x00000d19   Thumb Code     4  startup_hhd32f0xx_s.o(.text)
    NMI_Handler                              0x00000d1d   Thumb Code     2  startup_hhd32f0xx_s.o(.text)
    HardFault_Handler                        0x00000d1f   Thumb Code     2  startup_hhd32f0xx_s.o(.text)
    SVC_Handler                              0x00000d21   Thumb Code     2  startup_hhd32f0xx_s.o(.text)
    PendSV_Handler                           0x00000d23   Thumb Code     2  startup_hhd32f0xx_s.o(.text)
    SysTick_Handler                          0x00000d25   Thumb Code     2  startup_hhd32f0xx_s.o(.text)
    ADC_IRQHandler                           0x00000d27   Thumb Code     0  startup_hhd32f0xx_s.o(.text)
    BOD_IRQHandler                           0x00000d27   Thumb Code     0  startup_hhd32f0xx_s.o(.text)
    GPIOA_IRQHandler                         0x00000d27   Thumb Code     0  startup_hhd32f0xx_s.o(.text)
    GPIOB_IRQHandler                         0x00000d27   Thumb Code     0  startup_hhd32f0xx_s.o(.text)
    GPIOC_IRQHandler                         0x00000d27   Thumb Code     0  startup_hhd32f0xx_s.o(.text)
    PWM_FAULT_IRQHandler                     0x00000d27   Thumb Code     0  startup_hhd32f0xx_s.o(.text)
    PWM_TIMER_IRQHandler                     0x00000d27   Thumb Code     0  startup_hhd32f0xx_s.o(.text)
    RTC_IRQHandler                           0x00000d27   Thumb Code     0  startup_hhd32f0xx_s.o(.text)
    SPI_IRQHandler                           0x00000d27   Thumb Code     0  startup_hhd32f0xx_s.o(.text)
    TIMER16_0_IRQHandler                     0x00000d27   Thumb Code     0  startup_hhd32f0xx_s.o(.text)
    TIMER16_1_IRQHandler                     0x00000d27   Thumb Code     0  startup_hhd32f0xx_s.o(.text)
    TIMER16_2_IRQHandler                     0x00000d27   Thumb Code     0  startup_hhd32f0xx_s.o(.text)
    TIMER16_3_IRQHandler                     0x00000d27   Thumb Code     0  startup_hhd32f0xx_s.o(.text)
    TWS_IRQHandler                           0x00000d27   Thumb Code     0  startup_hhd32f0xx_s.o(.text)
    UART0_IRQHandler                         0x00000d27   Thumb Code     0  startup_hhd32f0xx_s.o(.text)
    UART1_IRQHandler                         0x00000d27   Thumb Code     0  startup_hhd32f0xx_s.o(.text)
    WAKEUP_IRQHandler                        0x00000d27   Thumb Code     0  startup_hhd32f0xx_s.o(.text)
    WDT_IRQHandler                           0x00000d27   Thumb Code     0  startup_hhd32f0xx_s.o(.text)
    __user_initial_stackheap                 0x00000d29   Thumb Code     0  startup_hhd32f0xx_s.o(.text)
    main                                     0x00000d49   Thumb Code    70  main.o(.text)
    AT24C02_ReadBYTE                         0x00000d9d   Thumb Code    14  at24c02.o(.text)
    AT24C02_WriteBYTE                        0x00000dab   Thumb Code    18  at24c02.o(.text)
    __aeabi_uidiv                            0x00000dbd   Thumb Code     0  aeabi_sdiv.o(.text)
    __aeabi_uidivmod                         0x00000dbd   Thumb Code    20  aeabi_sdiv.o(.text)
    __aeabi_idiv                             0x00000dd1   Thumb Code     0  aeabi_sdiv.o(.text)
    __aeabi_idivmod                          0x00000dd1   Thumb Code   326  aeabi_sdiv.o(.text)
    __use_two_region_memory                  0x00000f17   Thumb Code     2  heapauxi.o(.text)
    __rt_heap_escrow$2region                 0x00000f19   Thumb Code     2  heapauxi.o(.text)
    __rt_heap_expand$2region                 0x00000f1b   Thumb Code     2  heapauxi.o(.text)
    __user_setup_stackheap                   0x00000f1d   Thumb Code    62  sys_stackheap_outer.o(.text)
    exit                                     0x00000f5b   Thumb Code    12  exit.o(.text)
    __user_libspace                          0x00000f69   Thumb Code     8  libspace.o(.text)
    __user_perproc_libspace                  0x00000f69   Thumb Code     0  libspace.o(.text)
    __user_perthread_libspace                0x00000f69   Thumb Code     0  libspace.o(.text)
    _sys_exit                                0x00000f71   Thumb Code     8  sys_exit.o(.text)
    __I$use$semihosting                      0x00000f7d   Thumb Code     0  use_no_semi.o(.text)
    __use_no_semihosting_swi                 0x00000f7d   Thumb Code     2  use_no_semi.o(.text)
    __ARM_common_switch8                     0x00000f7f   Thumb Code    28  hhd_sys.o(i.__ARM_common_switch8)
    __semihosting_library_function           0x00000f7f   Thumb Code     0  indicate_semi.o(.text)
    Region$$Table$$Base                      0x00000f9c   Number         0  anon$$obj.o(Region$$Table)
    Region$$Table$$Limit                     0x00000fbc   Number         0  anon$$obj.o(Region$$Table)
    SystemCoreClock                          0x1000002c   Data           4  system_hhd32f0xx.o(.data)
    MainClock                                0x10000030   Data           4  system_hhd32f0xx.o(.data)
    __libspace_start                         0x10000034   Data          96  libspace.o(.bss)
    __temporary_stack_top$libspace           0x10000094   Data           0  libspace.o(.bss)



==============================================================================

Memory Map of the image

  Image Entry point : 0x000000c1

  Load Region LR_IROM1 (Base: 0x00000000, Size: 0x00000ff0, Max: 0x00016000, ABSOLUTE)

    Execution Region ER_IROM1 (Base: 0x00000000, Size: 0x00000fbc, Max: 0x00016000, ABSOLUTE)

    Base Addr    Size         Type   Attr      Idx    E Section Name        Object

    0x00000000   0x000000c0   Data   RO          137    RESET               startup_hhd32f0xx_s.o
    0x000000c0   0x00000008   Code   RO          259  * !!!main             c_p.l(__main.o)
    0x000000c8   0x0000003c   Code   RO          425    !!!scatter          c_p.l(__scatter.o)
    0x00000104   0x0000001a   Code   RO          427    !!handler_copy      c_p.l(__scatter_copy.o)
    0x0000011e   0x00000002   PAD
    0x00000120   0x0000001c   Code   RO          429    !!handler_zi        c_p.l(__scatter_zi.o)
    0x0000013c   0x00000002   Code   RO          297    .ARM.Collect$$libinit$$00000000  c_p.l(libinit.o)
    0x0000013e   0x00000004   Code   RO          310    .ARM.Collect$$libinit$$00000001  c_p.l(libinit2.o)
    0x00000142   0x00000000   Code   RO          314    .ARM.Collect$$libinit$$00000008  c_p.l(libinit2.o)
    0x00000142   0x00000000   Code   RO          316    .ARM.Collect$$libinit$$0000000A  c_p.l(libinit2.o)
    0x00000142   0x00000000   Code   RO          318    .ARM.Collect$$libinit$$0000000C  c_p.l(libinit2.o)
    0x00000142   0x00000000   Code   RO          321    .ARM.Collect$$libinit$$0000000F  c_p.l(libinit2.o)
    0x00000142   0x00000000   Code   RO          323    .ARM.Collect$$libinit$$00000011  c_p.l(libinit2.o)
    0x00000142   0x00000000   Code   RO          325    .ARM.Collect$$libinit$$00000013  c_p.l(libinit2.o)
    0x00000142   0x00000000   Code   RO          327    .ARM.Collect$$libinit$$00000015  c_p.l(libinit2.o)
    0x00000142   0x00000000   Code   RO          329    .ARM.Collect$$libinit$$00000017  c_p.l(libinit2.o)
    0x00000142   0x00000000   Code   RO          331    .ARM.Collect$$libinit$$00000019  c_p.l(libinit2.o)
    0x00000142   0x00000000   Code   RO          333    .ARM.Collect$$libinit$$0000001B  c_p.l(libinit2.o)
    0x00000142   0x00000000   Code   RO          335    .ARM.Collect$$libinit$$0000001D  c_p.l(libinit2.o)
    0x00000142   0x00000000   Code   RO          337    .ARM.Collect$$libinit$$0000001F  c_p.l(libinit2.o)
    0x00000142   0x00000000   Code   RO          339    .ARM.Collect$$libinit$$00000021  c_p.l(libinit2.o)
    0x00000142   0x00000000   Code   RO          341    .ARM.Collect$$libinit$$00000023  c_p.l(libinit2.o)
    0x00000142   0x00000000   Code   RO          345    .ARM.Collect$$libinit$$0000002A  c_p.l(libinit2.o)
    0x00000142   0x00000000   Code   RO          347    .ARM.Collect$$libinit$$0000002C  c_p.l(libinit2.o)
    0x00000142   0x00000000   Code   RO          349    .ARM.Collect$$libinit$$0000002E  c_p.l(libinit2.o)
    0x00000142   0x00000000   Code   RO          351    .ARM.Collect$$libinit$$00000030  c_p.l(libinit2.o)
    0x00000142   0x00000002   Code   RO          352    .ARM.Collect$$libinit$$00000031  c_p.l(libinit2.o)
    0x00000144   0x00000002   Code   RO          383    .ARM.Collect$$libshutdown$$00000000  c_p.l(libshutdown.o)
    0x00000146   0x00000000   Code   RO          410    .ARM.Collect$$libshutdown$$00000003  c_p.l(libshutdown2.o)
    0x00000146   0x00000000   Code   RO          413    .ARM.Collect$$libshutdown$$00000006  c_p.l(libshutdown2.o)
    0x00000146   0x00000000   Code   RO          416    .ARM.Collect$$libshutdown$$00000009  c_p.l(libshutdown2.o)
    0x00000146   0x00000000   Code   RO          418    .ARM.Collect$$libshutdown$$0000000B  c_p.l(libshutdown2.o)
    0x00000146   0x00000000   Code   RO          421    .ARM.Collect$$libshutdown$$0000000E  c_p.l(libshutdown2.o)
    0x00000146   0x00000002   Code   RO          422    .ARM.Collect$$libshutdown$$0000000F  c_p.l(libshutdown2.o)
    0x00000148   0x00000000   Code   RO          261    .ARM.Collect$$rtentry$$00000000  c_p.l(rtentry.o)
    0x00000148   0x00000000   Code   RO          267    .ARM.Collect$$rtentry$$00000002  c_p.l(rtentry2.o)
    0x00000148   0x00000006   Code   RO          279    .ARM.Collect$$rtentry$$00000004  c_p.l(rtentry4.o)
    0x0000014e   0x00000000   Code   RO          269    .ARM.Collect$$rtentry$$00000009  c_p.l(rtentry2.o)
    0x0000014e   0x00000004   Code   RO          270    .ARM.Collect$$rtentry$$0000000A  c_p.l(rtentry2.o)
    0x00000152   0x00000000   Code   RO          272    .ARM.Collect$$rtentry$$0000000C  c_p.l(rtentry2.o)
    0x00000152   0x00000008   Code   RO          273    .ARM.Collect$$rtentry$$0000000D  c_p.l(rtentry2.o)
    0x0000015a   0x00000002   Code   RO          302    .ARM.Collect$$rtexit$$00000000  c_p.l(rtexit.o)
    0x0000015c   0x00000000   Code   RO          356    .ARM.Collect$$rtexit$$00000002  c_p.l(rtexit2.o)
    0x0000015c   0x00000004   Code   RO          357    .ARM.Collect$$rtexit$$00000003  c_p.l(rtexit2.o)
    0x00000160   0x00000006   Code   RO          358    .ARM.Collect$$rtexit$$00000004  c_p.l(rtexit2.o)
    0x00000166   0x00000002   PAD
    0x00000168   0x00000400   Code   RO            3    .text               hhd_sys.o
    0x00000568   0x000002b4   Code   RO           53    .text               hhd_uart.o
    0x0000081c   0x0000048c   Code   RO           79    .text               hhd_iic.o
    0x00000ca8   0x00000070   Code   RO          108    .text               system_hhd32f0xx.o
    0x00000d18   0x00000030   Code   RO          138    .text               startup_hhd32f0xx_s.o
    0x00000d48   0x00000054   Code   RO          150    .text               main.o
    0x00000d9c   0x00000020   Code   RO          228    .text               at24c02.o
    0x00000dbc   0x0000015a   Code   RO          253    .text               c_p.l(aeabi_sdiv.o)
    0x00000f16   0x00000006   Code   RO          257    .text               c_p.l(heapauxi.o)
    0x00000f1c   0x0000003e   Code   RO          283    .text               c_p.l(sys_stackheap_outer.o)
    0x00000f5a   0x0000000c   Code   RO          286    .text               c_p.l(exit.o)
    0x00000f66   0x00000002   PAD
    0x00000f68   0x00000008   Code   RO          298    .text               c_p.l(libspace.o)
    0x00000f70   0x0000000c   Code   RO          353    .text               c_p.l(sys_exit.o)
    0x00000f7c   0x00000002   Code   RO          372    .text               c_p.l(use_no_semi.o)
    0x00000f7e   0x00000000   Code   RO          374    .text               c_p.l(indicate_semi.o)
    0x00000f7e   0x0000001c   Code   RO           19    i.__ARM_common_switch8  hhd_sys.o
    0x00000f9a   0x00000002   PAD
    0x00000f9c   0x00000020   Data   RO          423    Region$$Table       anon$$obj.o


    Execution Region RW_IRAM1 (Base: 0x10000000, Size: 0x00000398, Max: 0x00001000, ABSOLUTE)

    Base Addr    Size         Type   Attr      Idx    E Section Name        Object

    0x10000000   0x00000029   Data   RW           80    .data               hhd_iic.o
    0x10000029   0x00000003   PAD
    0x1000002c   0x00000008   Data   RW          109    .data               system_hhd32f0xx.o
    0x10000034   0x00000060   Zero   RW          299    .bss                c_p.l(libspace.o)
    0x10000094   0x00000004   PAD
    0x10000098   0x00000100   Zero   RW          136    HEAP                startup_hhd32f0xx_s.o
    0x10000198   0x00000200   Zero   RW          135    STACK               startup_hhd32f0xx_s.o


==============================================================================

Image component sizes


      Code (inc. data)   RO Data    RW Data    ZI Data      Debug   Object Name

        32          0          0          0          0        725   at24c02.o
      1164         74          0         41          0      13153   hhd_iic.o
      1052         54          0          0          0      30144   hhd_sys.o
       692         20          0          0          0      11873   hhd_uart.o
        84         14          0          0          0       1095   main.o
        48         22        192          0        768        752   startup_hhd32f0xx_s.o
       112         20          0          8          0       1099   system_hhd32f0xx.o

    ----------------------------------------------------------------------
      3186        204        224         52        768      58841   Object Totals
         0          0         32          0          0          0   (incl. Generated)
         2          0          0          3          0          0   (incl. Padding)

    ----------------------------------------------------------------------

      Code (inc. data)   RO Data    RW Data    ZI Data      Debug   Library Member Name

         8          0          0          0          0         68   __main.o
        60          8          0          0          0          0   __scatter.o
        26          0          0          0          0          0   __scatter_copy.o
        28          0          0          0          0          0   __scatter_zi.o
       346          0          0          0          0         92   aeabi_sdiv.o
        12          0          0          0          0         64   exit.o
         6          0          0          0          0        136   heapauxi.o
         0          0          0          0          0          0   indicate_semi.o
         2          0          0          0          0          0   libinit.o
         6          0          0          0          0          0   libinit2.o
         2          0          0          0          0          0   libshutdown.o
         2          0          0          0          0          0   libshutdown2.o
         8          4          0          0         96         68   libspace.o
         0          0          0          0          0          0   rtentry.o
        12          0          0          0          0          0   rtentry2.o
         6          0          0          0          0          0   rtentry4.o
         2          0          0          0          0          0   rtexit.o
        10          0          0          0          0          0   rtexit2.o
        12          4          0          0          0         60   sys_exit.o
        62          0          0          0          0         80   sys_stackheap_outer.o
         2          0          0          0          0         68   use_no_semi.o

    ----------------------------------------------------------------------
       618         16          0          0        100        636   Library Totals
         6          0          0          0          4          0   (incl. Padding)

    ----------------------------------------------------------------------

      Code (inc. data)   RO Data    RW Data    ZI Data      Debug   Library Name

       612         16          0          0         96        636   c_p.l

    ----------------------------------------------------------------------
       618         16          0          0        100        636   Library Totals

    ----------------------------------------------------------------------

==============================================================================


      Code (inc. data)   RO Data    RW Data    ZI Data      Debug   

      3804        220        224         52        868      58645   Grand Totals
      3804        220        224         52        868      58645   ELF Image Totals
      3804        220        224         52          0          0   ROM Totals

==============================================================================

    Total RO  Size (Code + RO Data)                 4028 (   3.93kB)
    Total RW  Size (RW Data + ZI Data)               920 (   0.90kB)
    Total ROM Size (Code + RO Data + RW Data)       4080 (   3.98kB)

==============================================================================

